:1000000000308A00512A00000A108A100A11820763
:1000100028340C34013406341A30840000080319E3
:10002000202801308D008C018C0B14288D0B132897
:100030004A308C008C0B1A2800000000800B11281D
:1000400000340608C339A100200D8C008C0DFC3053
:100050008C050C083C392104860006148316061012
:1000600000008312061083160610831200349E08C7
:10007000031D3C2886103D288614831686108312A3
:100080009F0E1F08A00021209F0E1F08A000212006
:100090000D308C008C0B4A28003414309A000C2050
:1000A000C33083168605831286108316861083124A
:1000B000061083160610831297011708023C031CD2
:1000C000692802309A000C200330A0002120970AF2
:1000D0005D280D308C008C0B6B280230A000212095
:1000E0000D308C008C0B722897011708023C031C02
:1000F00085281708042098009E0118089F003720C3
:1001000002309A000C20970A7528562A8E308C00EF
:100110001A088D0019088E008F018D08031D9A287A
:100120000E088D008E0108308C028D08031D9A2860
:100130008C01A22803108D1BA1288E0D8D0D8C0320
:100140009A288D1300003A29190803191529A100CE
:100150001D0803191529A107031CAF28B6287F30F5
:10016000A102031C152903191529BA288130A107FA
:100170000318152921088C008D018E018F011A08A2
:10018000A500A5171B08A4001C08A3001830A10097
:10019000A201231CE32820088F07031CD5288E0A00
:1001A000031DD5288D0A0319A2171F088E07031CEB
:1001B000DC288D0A0319A2171E089B009B171B0839
:1001C0008D070318A217A20D8D0C8E0C8F0CA50C99
:1001D000A40CA30C0310A10BC82801308C07031832
:1001E00015298D1BFA28A50D8F0D8E0D8D0D8C03F5
:1001F00003191529A51F0B298F0A031D0B298E0A28
:10020000031D0B298D0A031D0B298D0C8E0C8F0CE1
:100210008C0A031915291A08A2001E08A206A21F9B
:1002200013298D1719298D1319298C018D018E0120
:100230008F01000049291D308400FC308005800CAE
:10024000800C00080319282926290000800B252985
:10025000542918080F02031D322983160510831232
:100260000514362983168510831285149A01170800
:10027000990086289C019B017A309A00843099006D
:100280000F08A0000E089F000D089E000C089D009E
:10029000A4280C0899000D089A000E089B000F086E
:1002A0009C000C089D001B291808283C031D5D2993
:1002B0008316051083120510612983168510831299
:1002C00085100034831685158312851D622914302C
:1002D0008C008C0B69290000831685158312851903
:1002E000742900308D009829F9308C008C0B762908
:1002F00000000000831685158312851D83291A08C6
:100300008400800187291A0884000130800053305E
:100310008C008C0B89291A0884008008031D9229FF
:1003200005109329051483160510013083128D00E2
:100330000034170884008001013098001808043C3C
:10034000031CBE29170884000310000C8C008000D9
:1003500019309A0062218D08031DB12900308D00EB
:10036000C02917088400190D8C008C0D8C0DF830F5
:100370008C050C0800048000980A9E2901308D002D
:10038000003401301A029C001B08023C031DCA29DC
:1003900040309C071C0880389D009E011D089F006E
:1003A0003720003419088C000C300C020319E529A1
:1003B0000A300C020319ED290D300C020319F32940
:1003C00008300C020319F829FD299E0101309F0015
:1003D000372002309A000C20092A01309A0002309E
:1003E0009B00C121092A01309A009B00C121092AE2
:1003F0009E0110309F003720092A19081F3C031C5A
:10040000032A0730990501309E0019089F00372004
:10041000092A00341A088D0119020318122A190832
:100420008C001E2A8C0108309B00990D8C0D1A0837
:100430000C0203188C008D0D9B0B152A00340D083F
:100440001708990064309A000A220C0897000D08DA
:100450003030031D322A181898159819382A181A9E
:100460002030342A981118128D070D089900D221D6
:10047000170899000A309A000A220C0897000D0804
:100480003030031D472A98194B2A181A20308D073F
:100490000D089900D2213030970717089900D22112
:1004A000003484011F30830592014D2804309100EF
:1004B0001208970028309800292113089700293046
:1004C0009800292191010E309A0062218D08031DA8
:1004D0006A2A582A0E0B6E2A910A6F2A582A110886
:1004E000033C0318632A1430970099218D08031DDB
:1004F0007A2A582A1530970099218D08031D812AE0
:10050000582A1630970099218D08031D882A582AE9
:100510001608150203198D2A582A1408FD3E0318DF
:100520009E2A033ED32A15088F000F0892009E2AA8
:1005300015089000100893009E2A9E2A01309A0008
:100540009B00C12158309900D2213A309900D22124
:1005500020309900D2210F089700183098001F22F0
:100560000630970020309900D221970BB22A013033
:100570009A0002309B00C12159309900D2213A30B3
:100580009900D22120309900D2211008970018300C
:1005900098001F220630970020309900D221970B37
:1005A000CC2A562A63000A108A140A118207932A59
:0405B000982A9D2ABE
:02400E00F13F80
:00000001FF
